:020000040000FA
:0400000006303A2864
:08000800A000030EA100831209
:1000100005191028831601178312B23081002B288E
:1000200083160113831203140B190310A80DA90DD5
:10003000AA0DAB0DAC0DAC16FF302C02031D2B2806
:10004000FA302B02031D2B2831152A08AF0029088E
:10005000AE002808AD008B100B11210E8300A00EFE
:04006000200E090065
:0C007400203084008001840A6030040207
:10008000031C3C281230B00085218316FF2390000A
:10009000831283160C308505870183128501870141
:1000A000073099000030831691009F008312C830FA
:1000B00083168100831231309000003083168C004B
:1000C000831210308B00DD2181018E018F010B1115
:1000D0008B100B108C018B177B2031197E20B30BFA
:1000E0007928031085190314B90DF030390203196A
:1000F000FA20F1216C28640032100800311101301F
:10010000B7008B132030370783169B001C141A0886
:100110008312A4001030370783169B001C141A08A2
:100120008312A300A6000230A6060030370783160C
:100130009B001C141A088312A200A7000130A70616
:100140008B17321CA92822090339A200A309A4098C
:10015000A50924082F02031DF42823082E02031DDD
:10016000F42822082D02031DF42801303702031D54
:10017000BE283D18BE283D143E149321023037029C
:10018000031DC728BD18C728BD143E149A2103308B
:100190003702031DD0283D19D0283D153E14A1215A
:1001A00004303702031DD928BD19D928BD153E14C6
:1001B000A82105303702031DE2283D1AE2283D162A
:1001C0003E14AF2106303702031DEB28BD1AEB2881
:1001D000BD163E14B62107303702031DF4283D1B1F
:1001E000F4283D173E14BD21B70A08303702031822
:1001F000080081280130B600B300B400B500B70094
:1002000085018701B1137B20B30B382903108519B1
:100210000314B90DF030390203195F29B40B3829E2
:10022000013037020319C521023037020319C821F2
:10023000033037020319CB21043037020319CE21D2
:10024000053037020319D121063037020319D421B2
:10025000073037020319D7219630B4000330370234
:1002600032300319B4000430370232300319B400BD
:10027000311D03293111321C42292D090339AD00EA
:10028000AE09AF092F1C03298E018F010C1C032915
:100290000C102E1E03298B1320303707BB002F08AC
:1002A000BA00722110303707BB002E08BA00722145
:1002B00000303707BB002D08BA0072218B1785016B
:1002C0008701B70AB60108303702031C0329DD2174
:1002D00008003E1C08003E101030BB003D08BA006C
:1002E000722108008B133A0883161C159A003B08EC
:1002F0009B0055309D00AA309D009C1464009C1802
:100300007E291C1183128B170800831610309B0066
:100310001C141A088312BD00FF30D000D415D51567
:10032000D615D7150800BD103D11BD110230CE0005
:10033000D20008003D103D11BD110130CE00D200A9
:1003400008003D10BD10BD118230CE00D200080063
:100350003D10BD103D114130CE00D2000800BD124D
:100360003D13BD130030CF00D30008003D123D13F4
:10037000BD130230CF00D30008003D12BD12BD13E3
:100380000130CF00D30008000800013085060800C6
:100390000230850608000130850608000230850617
:1003A000080030308506080010308506080020302F
:1003B000850608002230850608003D189321BD18E7
:1003C0009A213D19A121BD19A8213D1AAF21BD1ABD
:1003D000B6213D1BBD21BD1BC4213D08031993213E
:1003E00008008F08031908008F0196308E00D00F87
:1003F000AB2AD00ABD1A232A521C232A521F142AC0
:10040000D41C052AD4015415312A541D0A2AD401BA
:10041000D415312AD41D0F2AD4015416312A541E62
:10042000312AD401D414312A541D192AD401541666
:10043000312AD41D1E2AD4015416312A541E312AC1
:10044000D401D414312AD41C282AD4015415312AB9
:10045000541D2D2AD401D415312A541E312AD40119
:100460005415BD1A5A2AD21C5A2AD21F4B2AD51CFF
:100470003C2AD5015515682A551D412AD501D515A7
:10048000682AD51D462AD5015516682A551E682AA0
:10049000D501D514682A551D502AD5015516682A4C
:1004A000D51D552AD5015516682A551E682AD5012D
:1004B000D514682AD51C5F2AD5015515682A551D03
:1004C000642AD501D515682A551E682AD501551507
:1004D000531C792A561D6F2AD6015616872AD61D17
:1004E000742AD6015616872A561E872AD601D61494
:1004F000872AD61C7E2AD6015615872A561D832A9E
:10050000D601D615872A561E872AD6015615D31C22
:10051000982A571D8E2AD7015716A62AD71D932A27
:10052000D7015716A62A571EA62AD701D714A62ADE
:10053000D71C9D2AD7015715A62A571DA22AD701D5
:10054000D715A62A571EA62AD701571569214E0886
:10055000D2004F08D3005008D1000C305405031DC1
:1005600085100C305505031D05100C305605031D74
:1005700085120C305705031D051251080E02031891
:10058000D52A12305405031D851412305505031D5C
:10059000051412305605031D851612305705031D2C
:1005A0000516FF305002031908008F08031D0800CC
:1005B0007B2051080E02031CD52A18305405031D58
:1005C000851006305405031D851418305505031D8C
:1005D000051006305505031D051418305605031D7A
:1005E000851206305605031D851618305705031D64
:0C05F000051206305705031D0516080013
:084000000E00030006000000A1
:02400E00CC01E3
:10420000010078007A007C007E007B0079007F004E
:104210007D007A0078007E007C00FF00FF00FF0038
:104220000000F200F600FA00FE00F200F600FA00CC
:10423000FE00F200F600FA00FE00FF00FF00FF00A3
:10424000010005000500050005000900090009003E
:1042500009000D000D000D000D00FF00FF00FF0024
:10426000FF00FF00FF00FF00FF00FF00FF00FF0056
:10427000FF00FF00FF00FF00FF00FF00FF00FF0046
:10428000FF00FF00FF00FF00FF00FF00FF00FF0036
:10429000FF00FF00FF00FF00FF00FF00FF00FF0026
:1042A000FF00FF00FF00FF00FF00FF00FF00FF0016
:1042B000FF00FF00FF00FF00FF00FF00FF00FF0006
:1042C000FF00FF00FF00FF00FF00FF00FF00FF00F6
:1042D000FF00FF00FF00FF00FF00FF00FF00FF00E6
:1042E000FF00FF00FF00FF00FF00FF00FF00FF00D6
:1042F000FF00FF00FF00FF00FF00FF00FF00DD00E8
:00000001FF
